:020000040000fa
:080000000406040000000000ea
:020000040000fa
:020000040002f8
:04afe000dfff00008f
:020000040000fa
:020000040002f8
:04afe400ffff00006b
:020000040000fa
:020000040002f8
:04afe80078ff0000ee
:020000040000fa
:020000040002f8
:04afec007dff0000e5
:020000040000fa
:020000040002f8
:04aff00078ff0000e6
:020000040000fa
:1000080000000000000000000000000000000000e8
:10001800fc050000000000000000000000000000d7
:10002800980a000000000000000000001a0b000001
:1000380000000000000000000000000000000000b8
:100048004c0b000000000000000000003e0c000007
:10005800b40c0000e00c00000000000000000000ec
:100068000000000000000000000000000000000088
:100078000000000000000000000000000000000078
:10008800000000000000000000000000780b0000e5
:100098000e0c00000000000000000000000000003e
:1000a8000000000000000000000000000000000048
:1000b8000000000000000000000000000000000038
:1000c8000000000000000000000000000000000028
:1000d8000000000000000000000000000000000018
:1000e8000000000000000000000000000000000008
:1000f80000000000000000000000000000000000f8
:1001080000000000000000000000000000000000e7
:1001180000000000000000000000000000000000d7
:1001280000000000800c000000000000000000003b
:1001380000000000000000000000000000000000b7
:1001480000000000000000000000000000000000a7
:100158000000000000000000000000000000000097
:100168000000000000000000000000000000000087
:100178000000000000000000000000000000000077
:100188000000000000000000000000000000000067
:100198000000000000000000480d0000740d000081
:1001a800a00d00000000000000000000000000009a
:1001b8000000000000000000000000000000000037
:1001c8000000000000000000000000000000000027
:1001d8000000000000000000000000000000000017
:1001e8000000000000000000000000000000000007
:1001f80000000000000000000000000000000000f7
:1002080000000000000000000000000000000000e6
:1002180000000000000000000000000000000000d6
:1002280000000000000000000000000000000000c6
:1002380000000000000000000000000000000000b6
:1002480000000000000000000000000000000000a6
:100258000000000000000000000000000000000096
:100268000000000000000000000000000000000086
:0c0278000000000000000000000000007a
:020000040000fa
:10040000803e2000030007008100e900fcff3a0065
:1004100000000600831f7800c20320000400bc0017
:1004200066015100e0815900f23fb1000380b10044
:1004300006003500ee03090000000000423fb10055
:100440000380b100fbff3d001200b000223fb0006e
:10045000020035000280090000000000cf01780092
:1004600000000600861f78006022b8000602200007
:100470000000d0008180d2000482d2008582d200a8
:100480000000a0000202520083825a0003003100e3
:100490000202420083824a000000a1000603e90034
:1004a000f3ff3a004f03780000000600f4ff2f002e
:1004b0000600070001003c000000050010000500d8
:1004c000140020000100370014002000889fbe00a7
:1004d0008a9fbe00841f7800730107004f007800d8
:1004e00011003300f0ff2f00838f6c0006003b00eb
:1004f000040565000a00a7000800370009f0a600ff
:100500001000200008003700820f5400838f5c0029
:10051000030039001000200001003e000000200010
:1005200009f0a7000000ea004f05be004f04be001e
:100530000000e000000006000002be00e00f5000d6
:10054000e08f5800020035002a0107000000060075
:100550000401be0061006100010020008301d100a0
:100560000281d30002007000838070002101070027
:100570000001be000100370003f0a200869fbe000c
:10058000889fbe008a9fbe008c9fbe004601070068
:10059000880133006450e1004f0032006420e10024
:1005a0005200320003826c0007003b000905d000b6
:1005b0000306d000820f54000c065d0002003900d3
:1005c0000200320089017800030678008582550018
:1005d00004003d000003fd008103fd008502ea00e8
:1005e0008b854200840f720002003b006000100007
:1005f000e08018006011b8000005eb007a28e100e7
:100600000a00390006007800c75ddd00f707b20078
:10061000878075002d003700828171000a01780003
:10062000610560008180d1000080d3008502e9006f
:10063000f9ff3b00060440008784480002003b00ad
:1006400060041400e0841c000988a3000700320045
:100650008a81710082817100610164008904d10086
:100660000884d3008b05e800170037000978a30041
:1006700013003a000b00e000130034008b05e90082
:100680000804440089844c000a4474000978a300db
:100690000d003a000b00e000070034008b05e90074
:1006a0000804440089844c0001003a000b0020003b
:1006b0000978a300f7ff32000001eb0002003700c9
:1006c000828171000a017800140107000cf0a70074
:1006d00001f0a000400137006420e10002003a0070
:1006e000838f6c00410133000801be000200be0090
:1006f00039013700869fbe00889fbe008a9fbe00da
:100700008c9fbe00e80007002a01330003866c00be
:100710006450e1002e0032006420e100330032001a
:100720006150e1002f0032006120e1003100320011
:1007300085855500eb07b000090020000804200063
:10074000050037000804440089844c000a00310089
:100750000603430087834b000001530081815b0047
:10076000f8ff33000203be000800a00008044400a4
:1007700089844c00f6ff3900c639dd00830173001f
:1007800001003200130020008904d1000884d30046
:100790000998a300050032000800a7000300a0008c
:1007a0008904d1000884d3008b05e8008904d100b6
:1007b0000884d3000001eb000281d200d7000700bb
:1007c00001f0a1000cf0a70001f0a0000201370029
:1007d0006420e100050132000801be000200be00f5
:1007e000f7ff37006120e100000132006000b8002f
:1007f000f3ff37000000200001f82700f0ff37006a
:10080000869fbe00889fbe008a9fbe008c9fbe0050
:10081000a5000700e700330003866c006450e10088
:10082000240032006420e100270032006150e10022
:10083000220032006120e100210032008b8542005d
:10084000eb07b1000134b800003ab80008044200d8
:1008500089844a00013ab8000030b800888040001e
:1008600009014a0004003300000040008180480074
:10087000020149008b05e900c909dd008301700010
:100880000100320013002000c814de004814dd000f
:100890004709de001200b200c808de0008847000bc
:1008a0009e00070001f0a1000cf0a70001f0a000dd
:1008b000c90037006120e100cc0032000801be0011
:1008c0000200be00f7ff37006150e100fcff3a0074
:1008d000c6003700829fbe000001be007a000700fc
:1008e0000470a70003f0a1006509b10018003200f0
:1008f0000e0035006828e10007003500f0ff2f00ea
:10090000f1ff27000300e00015003b000100280074
:100910004f01be000000050000004000818048003b
:100920008502e900fcff3a0009003700f88f420019
:1009300003003c008000eb004f01be0000000500fa
:100940008100d1000080d3008502e800fcff3a005e
:100950000300e00002003b0060001000e08018008f
:100960004f01be0000000600829fbe000001be00d5
:10097000550007000470a70003f0a10003f8a300ce
:1009800015003a006509b100110032000a00350077
:100990006928e10003003500010028004f01be0076
:1009a0000000050000004000818048008502e90049
:1009b000fcff3a0006003700f88f420006003500c1
:1009c0008100d1000080d3008502e800fcff3a00de
:1009d0004f01be00000006008000eb004f01be008a
:1009e000000005000000fb00cf80de0001003700a2
:1009f0008000eb00829fbe00889fbe008a9fbe00e1
:100a0000010578000100e0000400350008003c000a
:100a10000000e000200032000500370060001000f8
:100a2000e080180002003b0001f024001a003700ab
:100a30000004be006011b8006b0920000982cf00dd
:100a4000020039000882cf000441b0006942520020
:100a50000e00320008003b008281710061016400d9
:100a60008904d1000884d3008b05e8000442e80023
:100a7000f9ff3a00050037000804440089844c005f
:100a80008b05e9000442e900fbff3a002300070060
:100a90000af0a70001f0a0004f05be004f04be0001
:100aa0004f01be00000006000004be000600070063
:100ab0000003be000405be000200be0002000700e5
:100ac000844f750000000600c70ade00f107b2007f
:100ad000f50fb20008003200e1cf42000200320000
:100ae0000170a00024000500810f70000100320099
:100af0000408050044000500810f700002003a0060
:100b0000140005008502e9000000400081c0480093
:100b1000fcff3b000170a0002400050081002000c4
:100b2000618055000b003d000b00200061fe2f008e
:100b30000100e1001d003400828171006101640048
:100b40008904d1000884d3000000e800faff3a00cd
:100b5000710020006100640003007000020060006a
:100b60000900320061044400e0844c000988a500bb
:100b7000050032008b05e8006808e10002003a0039
:100b80008904d1000884d300f20f20000258e1004c
:100b900005003d00c75ddd00f907b20089807500e2
:100ba00008007800000006000bf827008b00780092
:100bb000000005000200be006450e10005003600a0
:100bc0006420e100020036000968a30001003a0039
:100bd0000800be000160a0004f06be004f05be0029
:100be0004f04be004f03be0000000600f0ff2f00c0
:100bf000f1ff2700f8ff37000020ef000220ef0090
:100c0000c088a900004006000f00210040272100f5
:100c100000018800000000000000eb0000077800e1
:100c20000c000900002f78000007eb005420ef00b3
:100c30000e2eef001e2eef000000eb0041272100da
:100c40008b1d09008018780040a7a900a100200092
:100c5000ebfd0700e0022000303a880044e7a900dd
:100c600044c7a9004407a9004427a9004447a90094
:100c70004467a9004487a900300020000600fc005a
:100c80003174200082072000a309200082487800e8
:100c90008348780080487800113a800061807000b5
:100ca0000600fc002174200062042000730520006f
:100cb0008248780083487800804878004427ef0015
:100cc000e0022000303a8800300020000d00fc00d7
:100cd0003174200082072000a30920008248780098
:100ce00083487800804878000000200021742000ac
:100cf0006204200073052000824878008348780051
:100d00008048780042a7ae00feff3700813e2000f9
:100d1000bbfd070010c0b30086e6b70090c2b30069
:100d2000c4e6b700000ea800007825008070880097
:100d300010cea900108ea90010aea900008ea90047
:100d4000100ea900102ea900002ea9004188a800ad
:100d500041a8a90041c8a90004a1a8000481a800d5
:100d600005e1a8000068a9000021ef0002a1ef0042
:100d70002068a8001061a8001021a90011e1a800b6
:100d800011a1a90010a1a8001081a8000821ef005e
:100d90000621ef000ca1ef000ea1ef004408a9000e
:100da0004428a9004448a9000108a9002108a80076
:100db0001fe1a8001fa1a9001ec1a9001ea1a80033
:100dc0001e81a8001e61a9001e21a9004d88a8004f
:100dd0004da8a8004dc8a900803e2000d00888007a
:100de0000368a9002368a80021e1a80021a1a900a7
:100df00020c1a90020a1a8002081a8002021a900cd
:100e00004e08a8004e28a9004e48a8000388a90053
:100e1000a00e2000e00888002388a8002002a90076
:100e20002022a9002042a90020a2a9002062a90036
:100e30002082a90020e2a9002102a9002122a90004
:100e4000700720004011880022a2a90022c2a90038
:100e500022e2a90021e2a8002182a9004588a90078
:100e600045a8a80045c8a8002168a8002828a8000f
:100e700023e2a9002342a8002362a9000188a90057
:100e80002188a8004608a9004628a8004648a800ce
:100e90000e0ea80021e3a9002143a80021a3a90068
:100ea0002123a9002103a90020e3a90020c3a90050
:100eb00020a3a9002083a9002043a80023e3a900c0
:100ec00023c3a90023a3a9002343a9002323a90026
:100ed0002303a90022c3a90022a3a9002283a900f9
:100ee0002263a9002243a9002223a9002203a9000a
:100ef0002563ef0024e3ef003223ef002823ef0007
:100f00002623ef002e23ef003023ef0021a8a800b6
:100f100046c8a80046a8a9004688a80001a8a900bc
:100f200021e3a8004008a9004028a9004048a800e3
:100f30002008a8000008a900c208a80080c0b300cb
:100f4000c8e8b7002bc8a9002be8a9002c08a90005
:100f50000bc8a9000be8a9000c08a90001eca90026
:100f600001aca900016ca900014ca900012ca90049
:100f7000010ca90000eca900008ca90000aca9009c
:100f800000cca900000ca900002ca900004ca9006d
:100f9000006ca900202cef00402cef00602cef002b
:100fa0000000210020608800020ca900022ca9008a
:100fb000024ca900262cef00462cef00662cef0017
:100fc000282cef00482cef00682cef000aacef0053
:100fd00023eca80023cca80023aca900238ca900f3
:100fe000236ca900234ca800232ca900230ca900e2
:100ff000222ca80043eca80043cca80043aca900d5
:10100000438ca900436ca800434ca900432ca900c1
:10101000430ca90063eca80063cca80063aca90052
:10102000638ca800636ca800634ca900dabc2a009a
:101030001b32240030002c00fa608800fb6088001e
:1010400020618800dabc2a001b32240020402c00da
:10105000fa608800fb60880010618800dabc2a0012
:101060001b32240030002c00fa608800fb608800ee
:1010700020628800dabc2a001b32240000802c0089
:10108000fa608800fb60880010628800dabc2a00e1
:101090001b32240030002c00fa608800fb608800be
:1010a00020638800dabc2a001b32240000802c0058
:1010b000fa608800fb60880010638800a700370092
:1010c0003f00370000202000006188000020200041
:1010d000006288000020200000638800020ca90044
:1010e000022ca800024ca80004acef0028acef00d2
:1010f00048acef0068acef00262cef00462cef0068
:10110000662cef000aacef0023eca80023cca9006a
:1011100043eca80043cca90063eca80063cca90071
:10112000dabc2a001b32240030002c00fa60880050
:10113000fb60880020618800dabc2a001b32240092
:1011400000002800fa608800fb60880010618800b9
:10115000dabc2a001b32240030002c00fa60880020
:10116000fb60880020628800dabc2a001b32240061
:1011700000002800fa608800fb6088001062880088
:10118000dabc2a001b32240030002c00fa608800f0
:10119000fb60880020638800dabc2a001b32240030
:1011a00000002800fa608800fb6088001063880057
:1011b00011eea90011aea900116ea9006700370059
:1011c000350037000010200000618800001020006a
:1011d000006288000010200000638800020ca90053
:1011e000022ca800024ca8000a2cef0004acef006f
:1011f000282cef005055250040628800a0aa2a0044
:1012000040638800dabc2a001b32240030002c0026
:10121000fa608800fb60880020618800dabc2a0040
:101220001b32240000002c00fa608800fb6088005c
:1012300010618800dabc2a001b32240030002c0028
:10124000fa608800fb60880020628800dabc2a000f
:101250001b32240000002c00fa608800fb6088002c
:1012600010628800dabc2a001b32240030002c00f7
:10127000fa608800fb60880020638800dabc2a00de
:101280001b32240000002c00fa608800fb608800fc
:101290001063880031003700300037000010200054
:1012a000006188000010200000628800020ca90084
:1012b000022ca800024ca8000a2cef0004acef009e
:1012c000282cef000000240040628800dabc2a00cd
:1012d0001b32240030002c00fa608800fb6088007c
:1012e00020618800dabc2a001b32240000002c0098
:1012f000fa608800fb60880010618800dabc2a0070
:101300001b32240030002c00fa608800fb6088004b
:1013100020628800dabc2a001b32240000002c0066
:10132000fa608800fb60880010628800dabc2a003e
:101330001b32240030002c00fa608800fb6088001b
:1013400020638800dabc2a001b32240000002c0035
:10135000fa608800fb60880010638800218ca90077
:10136000418ca900618ca900216ca900416ca900e5
:10137000616ca900214ca900414ca900614ca90055
:1013800020eca80040eca80060eca8003e2cef0088
:101390005e2cef007e2cef0001eca800d032ef00b5
:1013a000b232ef007b0a0700610b0700610c0700f7
:1013b000b4b2ef000000eb0041b62100ff030900ca
:1013c000805878008232ef008432ef00ee32ef0076
:1013d000f032ef000000eb0041f62100ff030900ae
:1013e000805878008632ef008832ef000080eb00f2
:1013f00081b421000d000900801878008e32ef00c2
:101400000000eb00e1332100ff00090080187800a4
:101410002a73ef002b73ef000000eb00e153210073
:10142000ff000900801878002d73ef000000eb002a
:10143000e1732100ff000900801878002e73ef008f
:101440002f73ef00f0c7b30030f3b7002000200087
:10145000f0c988002000200000ca88002000200079
:1014600010ca88002000200020ca88002000200028
:1014700030ca8800e432ef00e632ef00e832ef00d5
:10148000ea32ef00c232ef00f0c0b3003df3b70024
:10149000910c07002008a8002068a80021a8a80037
:1014a00001a8a9002003a9002023a8000012200001
:1014b000e00888000388a9002388a800803e200057
:1014c000d00888000368a9002368a800a832ef00ac
:1014d0000a33ef000c33ef00ce32ef00ca32ef00d8
:1014e000cc32ef0000c3b300b6f2b70040cab3007d
:1014f000b8f2b70020002000d095880010c0b300db
:10150000bcf2b700100020004096880010002000b8
:10151000309688000001200000968800c232ef005b
:1015200010002000b0968800f5050700aa013700da
:10153000ff3ffc004200f8003600f8004400f800cd
:101540008e1f78000e0020000d000900be1f7800dd
:101550003200f8007412f8007612f8000100fc0066
:101560000008a90000088000b0978800209580003e
:10157000c09788000021ef00a432ef00e02920008e
:1015800001002000d2978000e39780000201400014
:10159000838148000200be00b2978000c39780009c
:1015a000800f5100818f590010003600fa32ef0091
:1015b000fc32ef002e73ec00b2978000c3978000de
:1015c00080e2210051002000a6fb0700e13221004b
:1015d000914078008180fb0081804000e27321000f
:1015e00080307900a212a90005003700a212a800dd
:1015f000b0978000d0978800c0978000e09788005f
:10160000ff3ffc007612f9007412f9003200f90075
:10161000ae0120000d0009004f1778004f07780039
:101620004400f9003600f9004200f9000100fc0016
:1016300000400600ff3ffc004200f8003600f800c2
:101640004400f8008e1f78000e0020000d000900f5
:10165000be1f78003200f8000100fc000068a900fd
:101660000021ef00a432ec00a5f2a900ff3ffc002e
:101670003200f900ae0120000d0009004f1778007c
:101680004f0778004400f9003600f9004200f900e5
:101690000100fc0000400600ff3ffc004200f80093
:1016a0003600f8004400f8008e1f78000e0020007d
:1016b0000d000900be1f78003200f8000100fc0098
:1016c0000108a900ff3ffc003200f900ae01200034
:1016d0000d0009004f1778004f0778004400f9000b
:1016e0003600f9004200f9000100fc00004006004d
:1016f000ff3ffc004200f8003600f8004400f8000c
:101700008e1f78000e0020000d000900be1f78001b
:101710003200f8007412f8000100fc000368a90010
:101720001421ef002fd3bf002e53b50008003a005c
:101730002fd3bf000080fb0000004000e1732100b8
:1017400060807800f09788000033ef001e003700bb
:10175000fe32ef000033ef008c32ef002ed3bf00db
:101760002f53e3000e0032002f73ec008c32ec009c
:101770002fd3bf000080fb0000004000e173210078
:1017800060807800f297800003988000000041009c
:10179000e0804900f097880001988800efff37004b
:1017a0006294800001988000f39780001100090086
:1017b0008280d8008001fd00110009004288d80015
:1017c000f097880003988800800c2000010020001a
:1017d0007297800083978000020140008381480057
:1017e000c2da8800d3da88002913a800ff3ffc0082
:1017f0007412f9003200f900ae0120000d0009005a
:101800004f1778004f0778004400f9003600f900c0
:101810004200f9000100fc0000400600ff3ffc0010
:101820004200f8003600f8004400f8008e1f7800ef
:101830000e0020000d000900be1f78003200f800e5
:101840000100fc000388a9001821ef002023a90053
:10185000ff3ffc003200f900ae0120000d0009003e
:101860004f1778004f0778004400f9003600f90060
:101870004200f9000100fc0000400600ff3ffc00b0
:101880004200f8003600f8004400f8008e1f78008f
:101890000e0020000d000900be1f78003200f80085
:1018a0007812f8000100fc000168a9008212ec0027
:1018b00080007800f03f20000080600010948800d5
:1018c000129480003011800041b6210080707900b0
:1018d000ff3ffc007812f9003200f900ae01200051
:1018e0000d0009004f1778004f0778004400f900f9
:1018f0003600f9004200f9000100fc00004006003b
:10190000ff3ffc004200f8003600f8004400f800f9
:101910008e1f78000e0020000d000900be1f780009
:101920003200f8000100fc000828a9002242ae00a5
:10193000000037002222af002222a900ff3ffc0056
:101940003200f900ae0120000d0009004f177800a9
:101950004f0778004400f9003600f9004200f90012
:101960000100fc0000400600ff3ffc004200f800c0
:101970003600f8004400f8008e1f78000e002000aa
:101980000d000900be1f78003200f8000100fc00c5
:101990000188a900ff3ffc003200f900ae012000e1
:1019a0000d0009004f1778004f0778004400f90038
:1019b0003600f9004200f9000100fc00004006007a
:1019c000ff3ffc004200f8003600f8004400f80039
:1019d0008e1f78000e0020000d000900be1f780049
:1019e0003200f8000100fc0001a8a9002003a900b2
:1019f0000018800030958800409580003195800067
:101a0000808f50000400360040958000a612b5007b
:101a1000809588000300370030958000a812b5003b
:101a20008095880070958000b012b40060958800a1
:101a300080958000709588003095800040958800e2
:101a400080072000010020007297800083978000ab
:101a50000201400083814800a2da8800b3da8800de
:101a60002913a800ff3ffc003200f900ae0120005e
:101a70000d0009004f1778004f0778004400f90067
:101a80003600f9004200f9000100fc0000400600a9
:101a9000ff3ffc004200f8003600f8004400f80068
:101aa0008e1f78000e0020000d000900be1f780078
:101ab0003200f8000100fc000bc8a900ff3ffc0049
:101ac0003200f900ae0120000d0009004f17780028
:101ad0004f0778004400f9003600f9004200f90091
:101ae0000100fc0000400600ff3ffc004200f8003f
:101af0003600f8004400f8008e1f78000e00200029
:101b00000d000900be1f78003200f8000100fc0043
:101b10000be8a900ff3ffc003200f900ae012000f5
:101b20000d0009004f1778004f0778004400f900b6
:101b30003600f9004200f9000100fc0000400600f8
:101b4000ff3ffc004200f8003600f8004400f800b7
:101b50008e1f78000e0020000d000900be1f7800c7
:101b60003200f8000100fc000c08a900ff3ffc0057
:101b70003200f900ae0120000d0009004f17780077
:101b80004f0778004400f9003600f9004200f900e0
:101b90000100fc00004006001194800020948000a9
:101ba000808f50000a0032008412ec008000780020
:101bb000f03f200000806000209488002294800084
:101bc00040b62100604079001af3b70001003700e9
:101bd0001af3ef0000000600c15d200008fa0700bc
:101be0003008800070978800400880008097880047
:101bf0009083260021002000729780008397800048
:101c0000020140008381480042da880053da8800ec
:101c10003008800070978800400880008097880016
:101c20008e12af00090037009083260021002000ab
:101c300072978000839780000201400083814800f2
:101c400042da880053da88008e12a800d2ff07001b
:101c500050ccb3001a53b50006003900e0cfb300f2
:101c60001a53b50001003900010037001b73ef0063
:101c7000110137001af3ae00280037001b73ef0084
:101c800040c8b3001a53e30005003a001ad3bf005e
:101c90001bf3b7001cf3ef001df3ef001e0037002d
:101ca00040c9b3001a53e30005003a001ad3bf003d
:101cb0001bf3b7001ef3ef001ff3ef001600370011
:101cc00040cab3001a53e30005003a001ad3bf001c
:101cd0001bf3b70020f3ef0021f3ef000e003700f5
:101ce00040cbb3001a53e30005003a001ad3bf00fb
:101cf0001bf3b70022f3ef0023f3ef0006003700d9
:101d000040ccb3001a53e30003003a001ad3bf00db
:101d10001bf3b70024f3ef00e70037001b53e2008a
:101d200002003a00e4003700e300370040c8b30087
:101d30001b53e30026003a0000e0ef001c53e300d1
:101d400003003a001ad3bf001cf3b7001f0037008e
:101d50001ad3bf001df3b7001cd3bf00f1c2b300fc
:101d600080cf10000b003600b0c5b3001c53e30059
:101d700008003e0040c8b30038f3b7001cd3bf00d2
:101d800039f3b7001dd3bf003af3b7001d0a0700af
:101d90000d0037001cd3bf0071c7b30080cf100007
:101da00009003600e0c7b3001c53e30006003e0004
:101db00040c8b30038f3b7001cd3bf0039f3b700f5
:101dc0003a73ef000f0a07001cf3ef00ba00370068
:101dd00040c9b3001b53e30045003a0000e0ef00a8
:101de0001e53e30003003a001ad3bf001ef3b700ee
:101df0003e0037001ad3bf001ff3b7001f53e200a5
:101e00001c003a001ed3bf0071c7b30080cf100082
:101e10000a003600e0c7b3001e53e30007003e008f
:101e200040c9b30038f3b7001ed3bf0039f3b70081
:101e30003a73ef00f30907000d0037001ed3bf000f
:101e4000f1c2b30080cf100009003600b0c5b30066
:101e50001e53e30006003e0040c9b30038f3b7004c
:101e60001ed3bf0039f3b7003a73ef00e50907004e
:101e70001d0037001ed3bf0071c7b30080cf100014
:101e80000b003600e0c7b3001e53e30008003e001d
:101e900040c9b30038f3b7001ed3bf0039f3b70011
:101ea0001fd3bf003af3b700d60907000e00370072
:101eb0001ed3bf00f1c2b30080cf10000a0036006d
:101ec000b0c5b3001e53e30007003e0040c9b30095
:101ed00038f3b7001ed3bf0039f3b7001fd3bf00dc
:101ee0003af3b700c70907001ef3ef00720037008e
:101ef00040cab3001b53e30027003a0000e0ef00a4
:101f00002053e30003003a001ad3bf0020f3b700c8
:101f1000200037001ad3bf0021f3b70020d3bf0041
:101f200071c7b30080cf10000b003600e0c7b300cc
:101f30002053e30008003e0040cab30038f3b70066
:101f400020d3bf0039f3b70021d3bf003af3b70065
:101f5000ac0907000e00370020d3bf00f1c2b30068
:101f600080cf10000a003600b0c5b3002053e30054
:101f700007003e0040cab30038f3b70020d3bf00cb
:101f800039f3b70021d3bf003af3b7009d0907002a
:101f900020f3ef004800370040cbb3001b53e300b1
:101fa0000a003a0000e0ef002253e30003003a0089
:101fb0001ad3bf0022f3b700030037001ad3bf00c3
:101fc00023f3b700470207003b00370040ccb300c3
:101fd0001b53e30038003a0000e0ef002453e30015
:101fe00035003a001ad3bf0024f3b70030c0b30065
:101ff0002453e30006003e0040ccb3003bf3b7009f
:1020000024d3bf003cf3b7009e0907002900370026
:1020100024d3bf00f1c0b30080cf100025003600ec
:1020200030c1b3002453e30022003e0000c1b300de
:102030002473b500b232ef00c232ef002453e20045
:1020400002003a002e0307001700370024d3bf0018
:1020500080407800e1cf500002003a0043030700bf
:102060001100370024d3bf0080407800e2cf500039
:1020700002003a009b0607000b00370024d3bf0084
:1020800080407800e3cf500002003a005803070078
:102090000500370024d3bf0080407800e4cf500013
:1020a00001003a006c06070024d3bf003df3b700df
:1020b0008909070024f3ef000bc1bf00cdd2b600a1
:1020c0001040b20004003200cd12a8000b01ae0097
:1020d000cd12a900de32ec00c212e20048003a0044
:1020e000d012e2000c003a00f096800011978000b8
:1020f000808f5000020036006003070005003700a3
:10210000de32ef00b232ef001803070010002000ab
:10211000809688003a00370081968000e18f500059
:102120000c003a00f096800011978000808f5000dc
:10213000020036003b04070005003700de32ef00e6
:10214000b232ef006706070020002000809688006a
:102150002b00370081968000e28f50000c003a007f
:10216000f096800011978000808f500002003600aa
:102170007f06070005003700de32ef00b232ef00c5
:102180001b03070030002000809688001c003700e9
:1021900081968000e38f50000c003a00f09680009a
:1021a00011978000808f500002003600ce04070097
:1021b00005003700de32ef00b232ef0026060700de
:1021c00040002000809688000d0037008196800036
:1021d000e48f50000a003a00f096800011978000ca
:1021e000808f50000200360072050700040037009f
:1021f000de32ef00b232ef00c1020700d032ef0052
:102200002913af009a01070070c0b3002853b5002e
:10221000560131007297800083978000909780006c
:10222000a1978000800f5100818f59002e01390045
:10223000f5f2a8002853e2000f003a003097800022
:1022400020978800e632ef00509780004097880082
:10225000ea32ef0090832600210020007297800070
:1022600083978000020140008381480042da8800a1
:1022700053da88001b01370028d3bf008040780064
:10228000e1cf50000c003a003553e2000700360061
:1022900040c8b30038f3b70035d3bf0039f3b700f7
:1022a0003a73ef00d70807003573ef004cbbef001f
:1022b0004ebbef000b01370028d3bf0080407800f1
:1022c000e2cf500003003a0050bbef0052bbef00da
:1022d0000401370028d3bf0080407800e3cf5000ce
:1022e00053003a003298800043988000d0cc2c00f4
:1022f000c1f6230042f90700c0938800d1938800fb
:1023000060958000baf907000001be00a09929007d
:1023100091d923003af90700c2938000d39380003b
:1023200096f8070030988800419888002a73ec00de
:102330003098800041988000020020000320240093
:10234000ecf8070088f90700a132210091407800dd
:102350008180fb0081804000e233210080307900e1
:102360002ad3bf000080fb0000004000e1332100c1
:1023700060807800a09388002ad3bf008080fb0093
:10238000b8d2bf000080fb00008650000c0646005b
:10239000e033210060007e007412b50092f907005e
:1023a000c0938800d1938800b8d2bf008df9070090
:1023b0000001be00c0938000d1938000cdf80700db
:1023c00070988800819888002ad3bf000080fb00a5
:1023d00000004000e1332100608078004500dd000e
:1023e000306388002ad3bf000080fb00000040005b
:1023f000e133210060807800800078003097800011
:10240000808f5000060034002ad3bf000080fb00fc
:1024100000004000e13321006080780030978800a0
:1024200054bbef0056bbef002c13a800ad003700e3
:1024300028d3bf0080407800e4cf50009a003a00d3
:1024400012988000239880000000200001f42300ef
:10245000ebf80700c0938800d1938800f0978000c4
:102460000198800034f807000001be000000200041
:1024700001e82300e2f80700c2938000d3938000b4
:102480003ef8070010988800219888002d73ec0012
:102490002ad3bf000080fb0000004000e133210090
:1024a00060807800a0938800bcd2bf008000fb0051
:1024b000a0938000808f500028003c00109880007e
:1024c0002198800003f90700801f78002dd3bf00fa
:1024d0000081fb0002014100e15321004fb178006f
:1024e0002dd3bf008080fb00b6d2bf000080fb0070
:1024f000008650000c064600e053210060007e007c
:1025000039f907000001be00109880002198800072
:1025100019f80700c0938800d1938800b6d2bf0095
:1025200030f907000001be00c0938000d193800005
:1025300070f80700509888006198880052988000d1
:10254000639880000096800029f90700acf8070026
:10255000e0f80700709688002e0037002dd3bf00ea
:102560000080fb000006e9000c064600e053210055
:1025700060007e004180de00d13221009140780071
:102580008180fb0081804000e2532100803079008f
:102590002dd3bf000080fb0000004000e15321006c
:1025a00060807800a09388002dd3bf008080fb005e
:1025b000b6d2bf000080fb00008650000c0646002b
:1025c000e053210060007e007412b50006f9070098
:1025d000c0938800d1938800b6d2bf0001f90700ec
:1025e0000001be00c0938000d193800041f8070035
:1025f0005098880061988800529880006398800005
:1026000000968000faf807007df80700b1f807008f
:10261000709688002dd3bf000080fb0000004000b2
:10262000e1532100608078008000780010082000cd
:10263000808f500008003c002dd3bf000080fb00bd
:1026400000004000e1532100608078004500dd007b
:102650003062880002003700f0ff200030618800ff
:102660002dd3bf000080fb0000004000e15321009b
:10267000608078008000780050978000808f500044
:10268000060034002dd3bf000080fb000000400096
:10269000e1532100608078005097880058bbef001c
:1026a0005abbef000f00370028d3bf0080407800ee
:1026b000e5cf500004003a008eb2a9005cbbef00e9
:1026c0005ebbef000700370028d3bf0080407800d2
:1026d000e6cf500003003a008ed2a90060bbef00a5
:1026e00062bbef0062000700f1f2ae001e0037008f
:1026f0000821ef000621ef00ee32ef00f032ef008c
:102700000080eb0081b421000d00090080187800e2
:102710009083260040da88002000200050da8800ec
:1027200080072000a0da8800563bef00800c2000d4
:10273000c0da88005a3bef002913a800e0c0b300bc
:102740003df3b700e407070040cbb30038f3b70010
:10275000b0c7b30039f3b7003a73ef00a907070019
:10276000d032ef002afd370009003700f1f2ae0049
:10277000070037000821ef000621ef00ee32ef00de
:10278000f032ef00d0c0b3003df3b700d20707002e
:102790004194800030948000808f500010003200ff
:1027a0000188af000e0037002302ae000c00370096
:1027b0008812ec0080007800f03f2000008060006c
:1027c000409488004294800040f6210060407900e7
:1027d0000080fb0020118800001420000df7070086
:1027e000128eaa00108ea900f012af0014cea8001d
:1027f000f012ae0014cea9002c13ae001b0037005f
:102800002ad3bf000080fb0000004000e13321001c
:10281000608078008000780030d3bf000000fb00ab
:10282000810f5000060034002ad3bf000080fb0057
:1028300000004000e133210060c0780030f3b700b1
:1028400030d3bf000080fb000020ec008000780047
:10285000bcd2bf000080fb00810f5000020031009d
:102860003053ec00bcf2b7002c13a900e8fc370091
:1028700028f3ef00f5f2a8008a32ef0050948000b0
:10288000c200dd0080b42100008040001000be00c6
:102890000001be0090978000a1978000800f51003a
:1028a000818f59000900310050948000c200dd0082
:1028b00080b42100008040001000be009097880086
:1028c000a19788008ad2bf0028f3b7008a32ec00b3
:1028d00051948000e78f5000e8ff3a002913a900c7
:1028e0000000060022d3bf0080407800f7cf5000e0
:1028f00008003a0040cbb30038f3b70070c1b30012
:1029000039f3b70023d3bf003af3b7003d07070000
:10291000f900370022d3bf00d1c1b30080cf10002f
:102920000b00360090c2b3002253e30008003e00c3
:1029300040cbb30038f3b70022d3bf0039f3b70060
:1029400023d3bf003af3b7002e070700ea00370091
:1029500022d3bf0011c3b30080cf10000b0036009c
:10296000d0c3b3002253e30008003e0040cbb300c5
:1029700038f3b70022d3bf0039f3b70023d3bf0029
:102980003af3b7001f070700db00370000c4b300ad
:102990002253b5000300320010c4b3002253e300f9
:1029a00008003a0040cbb30038f3b70022d3bf0091
:1029b00039f3b70023d3bf003af3b700110707007c
:1029c000cd00370020c4b3002253e3002c003a00ae
:1029d00040cbb30038f3b70020c4b30039f3b700dd
:1029e00023d3bf003af3b700060707002353e200e2
:1029f00022003a008a32ef0051948000e68f5000a6
:102a00000a003e0050948000c200dd0080b4210026
:102a100000814000f0ff2f00f1ff2f000089be0071
:102a20008e32ef008a32ec00f3ff39002913a80040
:102a3000b232ef0000c3b300b6f2b70040cab30031
:102a4000b8f2b70020002000d095880010c0b30075
:102a5000bcf2b70010002000409688001000200053
:102a6000309688000001200000968800f0072000c2
:102a70001096880010002000b09688009e00370055
:102a800060c4b3002253e3000a003a0023d3bf001e
:102a90000080fb0000004000c09388007852ec00ea
:102aa000b6f2b700c09380001040b000b6f2b70095
:102ab0009100370070c4b3002253e3000a003a00cb
:102ac00023d3bf000080fb0000004000c0938800bb
:102ad0007852ec00b8f2b700c09380001040b0000c
:102ae000b8f2b7008400370090c4b3002253e3006b
:102af00004003a0023d3bf000080fb00d09588007b
:102b00007d003700a0c4b3002253e30003003a0065
:102b100023d3bf00bcf2b70077003700d0c4b300a6
:102b20002253e30005003a0023d3bf000080fb00de
:102b30000020ec00f09588006f003700e0c4b3007f
:102b40002253e30005003a0023d3bf000080fb00be
:102b50000020ec000096880067003700f0c4b30046
:102b60002253e3000c003a0023d3bf000080fb0097
:102b700010968800c212e2000600360040cbb30077
:102b800038f3b700b0c7b30039f3b7003a73ef00ba
:102b90009c0607005800370022d3bf00f1c4b300e1
:102ba00080cf10000b003600b0c5b3002253e30005
:102bb00008003e0040cbb30038f3b70022d3bf007b
:102bc00039f3b70023d3bf003af3b7008d060700ef
:102bd0004900370022d3bf0031c6b30080cf1000b8
:102be0000b003600f0c6b3002253e30008003e009d
:102bf00040cbb30038f3b70022d3bf0039f3b7009e
:102c000023d3bf003af3b7007e0607003a0037002f
:102c100000c7b3002253e3000b003a00f0c7b30033
:102c20002353b5000500310023d3bf000080fb0013
:102c30004500dd003061880002003700f0ff200011
:102c4000306188002c00370020c7b3002253e30016
:102c500004003a0023d3bf000080fb00f0c98800c5
:102c60002500370030c7b3002253e30004003a00c8
:102c700023d3bf000080fb0000ca88001e0037007d
:102c800040c7b3002253e30004003a0023d3bf003f
:102c90000080fb0010ca88001700370050c7b3003f
:102ca0002253e30004003a0023d3bf000080fb005e
:102cb00020ca88001000370060c7b3002253e30029
:102cc00004003a0023d3bf000080fb0030ca880014
:102cd00009003700b0c7b3002253e30006003a00f2
:102ce00040cbb30038f3b700b0c7b30039f3b70037
:102cf0003a73ef004306070022f3ef0000000600de
:102d000040cbb30038f3b70020c4b30039f3b700a9
:102d100050c5b3003af3b7003a06070040cbb30002
:102d200038f3b70000c4b30039f3b7003a73ef00cb
:102d300034060700b2b2ef00100020004096880071
:102d40001000200030968800d032ef00f09680000e
:102d500000978800f0c98000e012b4001097880046
:102d6000b432ef003d73ef005b06370040cbb30099
:102d700038f3b70020c4b30039f3b70050c5b3002f
:102d80003af3b7001f06070040cbb30038f3b70093
:102d9000b0c7b30039f3b7003a73ef001906070064
:102da00040cbb30038f3b70000c4b30039f3b70029
:102db00000c4b3003af3b70012060700b2b2ef0046
:102dc000100020008096880010002000b096880037
:102dd000f09680000097880000ca8000e012b400de
:102de0001097880010c0b3003df3b7003a063700d3
:102df00040cbb30038f3b70020c4b30039f3b700b9
:102e000050c5b3003af3b700fe05070040cbb3004e
:102e100038f3b700b0c7b30039f3b7003a73ef0027
:102e2000f805070040cbb30038f3b70000c4b30087
:102e300039f3b70000c4b3003af3b700f105070057
:102e4000b2b2ef0030002000809688001000200011
:102e5000b0968800f09680000097880020ca800015
:102e6000e012b40010978800b0022000209688007d
:102e700030c0b3003df3b70017063700b212e200ce
:102e800001003a009eff070001002000f072af0031
:102e90001140b000cc12af001140b10077003200f9
:102ea000cc12a800f072ae00cc12a9002dd3bf0046
:102eb0000080fb0000004000e153210060807800aa
:102ec000a093880032968000a09380000200e0006a
:102ed00002003200110009000200d800209688008c
:102ee00021968000eb8f500003003600c632ec00c4
:102ef000b0002000209688002296800040362200f4
:102f00006040790032f3b7002ad3bf000080fb0095
:102f100000004000e133210060c0780036f3b700c4
:102f2000bcd2bf003653e3001800360033d3bf00d5
:102f30003253e3000900320040c9b30038f3b70050
:102f400032d3bf0039f3b70036d3bf003af3b7002e
:102f5000ac05070032d3bf0033f3b7000df3ae006a
:102f600009003700ca32ae000700370040c8b3007e
:102f700038f3b700e0c7b30039f3b7003a73ef0096
:102f8000a0050700ca32a900130037003353e2003e
:102f90000700360040c8b30038f3b70033d3bf0092
:102fa00039f3b7003a73ef00960507003373ef006b
:102fb000ca32af000800370040c9b30038f3b70089
:102fc000e0c7b30039f3b700f0c7b3003af3b70076
:102fd0008c050700ca32a800a212ae001500370007
:102fe000ca52af000800370040c9b30038f3b70039
:102ff000c0c7b30039f3b700f0c7b3003af3b70066
:1030000080050700ca52a800ca72af000800370046
:1030100040c9b30038f3b700d0c7b30039f3b700e5
:10302000f0c7b3003af3b70076050700ca72a800ec
:1030300012003700ca52ae000700370040c8b30084
:1030400038f3b700c0c7b30039f3b7003a73ef00e5
:103050006c050700ca52a900ca72ae00070037000b
:1030600040c8b30038f3b700d0c7b30039f3b70096
:103070003a73ef0063050700ca72a900f0d2bf00df
:10308000ccd2b6004040b2001d003200cc52a800a5
:10309000f052ae00cc52a900729880008398800054
:1030a0000000200001f8230007f507000b003d0099
:1030b000ca12af000800370040c9b30038f3b700a8
:1030c000b0c7b30039f3b700f0c7b3003af3b700a5
:1030d0004c050700ca12a80009003700ca12ae004a
:1030e0000700370040c8b30038f3b700b0c7b300db
:1030f00039f3b7003a73ef0042050700ca12a9007e
:1031000001002000f092af001140b000cc32af00bf
:103110001140b10042003200cc32a800f092ae0063
:10312000cc32a9002dd3bf000080fb00000040007e
:10313000e153210060807800a093880042968000cf
:10314000a09380000200e00002003200110009009c
:103150000200d8002096880021968000b00220004e
:10316000808f500003003600c832ec00b00220000f
:103170002096880022968000003722006040790067
:1031800034f3b7002ad3bf000080fb0000004000ea
:10319000e133210060c0780036f3b700bcd2bf0035
:1031a0003653e3001500360035d3bf003453e30037
:1031b000110032003553e2000600360040c8b3006b
:1031c00038f3b70035d3bf0039f3b7003a73ef00d7
:1031d0000c05070040c9b30038f3b70034d3bf0073
:1031e00039f3b70036d3bf003af3b700050507003f
:1031f00034d3bf0035f3b700090037003553e20080
:103200000700360040c8b30038f3b70035d3bf001d
:1032100039f3b7003a73ef00fa0407003573ef0093
:1032200000000600b212e20001003a00cffe0700e3
:103230008eb2af00a20037007098800081988000a5
:10324000020020000300200098f40700801f78008f
:103250005098800061988000020020000300200048
:1032600092f407004f006000160032009298800030
:10327000a39880006066260061f6230060f50700d1
:10328000c0938800d1938800709880008198800056
:10329000529880006398800059f507000001be0035
:1032a000d0cc2c00c1dc230055f50700c293800070
:1032b000d3938000b1f4070090988800a19888000b
:1032c0000700370090988000a1988000020020003d
:1032d0000308240007f5070090988800a19888004b
:1032e000ec32ef0092988000a3988000d095800087
:1032f000bff5070074f4070003003d001000200034
:103300006097880001003700ec32ef002ad3bf003d
:103310000080fb0000004000e13321006080780065
:10332000a0938800bcd2bf008000fb00a093800067
:10333000808f500001003d00ec32ec00619780006e
:10334000e28f500049003a00b0968000a8f50700cf
:103350000001be0090988000a1988000e5f407006d
:1033600081f50700a0968800a1968000ec8f5000a0
:1033700003003600d632ec00c0002000a096880082
:10338000a0968000e00f500002003e0010002000d8
:10339000a0968800a0968000c412b40020968800f1
:1033a00021968000b0022000808f5000010036007e
:1033b000c432ef002296800000372200604079007e
:1033c00034f3b700e4d2bf0036f3b70040c9b3000e
:1033d00038f3b70034d3bf0039f3b70036d3bf009a
:1033e0003af3b7008704070034d3bf0035f3b700c2
:1033f0008eb2a800409780005094880051948000bd
:10340000f0072000808f500002003600f0072000f7
:103410005094880052948000020141008094210061
:1034200060007900010020004409dd00cc00de00ce
:10343000810071004400dd00b0988800c1988800c8
:10344000b0988000c19880007297800083978000b8
:1034500002004000838048000001be00e2da8800dc
:10346000f3da88002913a800140037003553e2006e
:103470000800360040cbb30038f3b700b0c7b30044
:1034800039f3b7003a73ef005e0407003573ef00bd
:103490000a003700ca52af000800370040c9b30025
:1034a00038f3b700c0c7b30039f3b700e4d2bf00a8
:1034b0003af3b70053040700ca52a80009003700c6
:1034c000ca52ae000700370040c8b30038f3b70057
:1034d000c0c7b30039f3b7003a73ef0049040700df
:1034e000ca52a90000000600b212e20001003a0030
:1034f0003ffe07008eb2af00a40037007098800036
:10350000819880000200200003002000e7f30700fc
:10351000801f780050988000619880000200200091
:1035200003002000e1f307004f00600016003200a6
:1035300092988000a39880006066260061f62300c0
:10354000aff40700c0938800d19388007098800082
:10355000819880005298800063988000a8f407004a
:103560000001be00d0cc2c00c1dc2300a4f4070075
:10357000c2938000d393800000f4070090988800e5
:10358000a19888000700370090988000a1988000db
:10359000020020000308240056f4070090988800d9
:1035a000a1988800ec32ef0092988000a3988000e8
:1035b000d09580000ef50700c3f3070003003d001f
:1035c000100020006097880001003700ec32ef0007
:1035d0002ad3bf000080fb0000004000e13321003f
:1035e00060807800a0938800bcd2bf008000fb0000
:1035f000a0938000808f500001003d00ec32ec0071
:1036000061978000e28f50004b003a00b096800036
:10361000f7f407000001be0090988000a198800098
:1036200034f40700d0f40700a0968800a19680002b
:10363000ec8f500003003600d632ec00c0002000b2
:10364000a0968800a0968000e00f500002003e0087
:1036500010002000a0968800a1968000209680008f
:10366000808f500004003e00a0968000c412b50078
:103670002096880002003700b002200020968800c3
:1036800022968000003722006040790034f3b700b2
:10369000e4d2bf0036f3b70040c9b30038f3b70037
:1036a00034d3bf0039f3b70036d3bf003af3b700c5
:1036b000d403070034d3bf0035f3b7008eb2a8009f
:1036c000409780005094880051948000f0072000bb
:1036d000808f500002003600f007200050948800d0
:1036e0005294800002014100809421006000790022
:1036f000010020004409dd00cc00de0081007100e3
:103700004400dd00b0988800c1988800b09880001f
:10371000c19880007297800083978000020040006b
:10372000838048000001be00e2da8800f3da8800f6
:103730002913a800140037003553e20008003600b2
:1037400040cbb30038f3b700b0c7b30039f3b700cc
:103750003a73ef00ab0307003573ef000a00370040
:10376000ca72af000800370040c9b30038f3b70091
:10377000d0c7b30039f3b700e4d2bf003af3b700c3
:10378000a0030700ca72a80009003700ca72ae0081
:103790000700370040c8b30038f3b700d0c7b30004
:1037a00039f3b7003a73ef0096030700ca72a90015
:1037b00000000600b212e20004003a00a600070072
:1037c000cc12a800f012ae00cc12a900f0d2bf00bb
:1037d000ccd2b6001040b20084003200cc12a80057
:1037e000f012ae00cc12a900e0968000d2968000c4
:1037f0000200e00002003200110009000280d8003f
:10380000e0968800da32ef002ad3bf000080fb0088
:1038100000004000e133210060807800a093880020
:10382000bcd2bf008000fb00a0938000808f5000be
:103830005a003d000df3af0039003700e1968000db
:1038400020968000808f50002b003200e096800090
:103850002096880021968000b0022000808f5000c2
:1038600008003600c20020002096800011000900e8
:103870000280d800c1938800b00220007812b40002
:1038800020968800209680004106de000037220046
:1038900060407e0034f3b70034d3bf003553e300fb
:1038a000140032003553e2000700360040c8b30070
:1038b00038f3b70035d3bf0039f3b70000c6b30003
:1038c0003af3b7004f03070034d3bf0035f3b70016
:1038d000e4d2bf0036f3b70040c9b30038f3b700f5
:1038e00034d3bf0039f3b70036d3bf003af3b70083
:1038f0004403070009003700ca32ae000700370052
:1039000040c8b30038f3b700e0c7b30039f3b700dd
:103910003a73ef003b030700ca32a9001e003700cc
:103920000200200003f82b0050988000619880006e
:10393000e3f2070018003c003553e20008003600af
:1039400040c8b30038f3b70035d3bf0039f3b70030
:1039500000c4b3003af3b7002a0307003573ef0041
:10396000ca32af000c00370040c9b30038f3b700cb
:10397000e0c7b30039f3b7002ad3bf000080fb00d3
:1039800000004000e133210060c078003af3b70046
:103990001c030700ca32a800090037003553e200b3
:1039a0000700360040cbb30038f3b700b0c7b30010
:1039b00039f3b7003a73ef00120307003573ef00d5
:1039c000dc32ef00ca12ae000700370040c8b30077
:1039d00038f3b700b0c7b30039f3b7003a73ef005c
:1039e00008030700ca12a9001a003700c196800018
:1039f0002dd3bf000080fb00810f50000b00320070
:103a00002dd3bf000080fb0000004000e1532100e7
:103a100060807800dc12b400e09688002dd3bf00ef
:103a20000080fb00c0968800da32ec00ca12af00ba
:103a30000800370040c9b30038f3b700b0c7b3007f
:103a400039f3b70000c4b3003af3b700ed02070042
:103a5000ca12a8000000060040cbb30038f3b7003c
:103a600020c4b30039f3b70050c5b3003af3b70030
:103a7000e402070040cbb30038f3b700b0c7b3008f
:103a800039f3b7003a73ef00de02070040cbb30012
:103a900038f3b70000c4b30039f3b7003a73ef004e
:103aa000d8020700b2b2ef00c432ef00400020009d
:103ab00080968800f09680000097880030ca8000c9
:103ac000e012b4001097880010002000d096880003
:103ad000d832ef00dc32ef0040c0b3003df3b70056
:103ae000fd02370040cbb30038f3b70020c4b30069
:103af00039f3b70050c5b3003af3b700c10207006d
:103b000040cbb30038f3b700b0c7b30039f3b70008
:103b10003a73ef00bb02070040cbb30038f3b700a5
:103b200000c4b30039f3b700f0c7b3003af3b700ed
:103b3000b4020700b2b2ef00200020008096880097
:103b4000f0968000009788001000200040968800c2
:103b5000100020003096880010ca8000e012b400e7
:103b60001097880020c0b3003df3b700da02370099
:103b7000b212e20001003a00daff07000100200063
:103b8000f032af001140b000cc12af001140b100d4
:103b90005c003200cc12a800f032ae00cc12a900ba
:103ba0002dd3bf000080fb0000004000e153210046
:103bb00060807800a093880042968000a0938000e7
:103bc0000200e00002003200110009000200d800eb
:103bd0002096880021968000b0022000808f50003f
:103be00003003600c832ec00b002200020968800a6
:103bf00022968000003722006040790034f3b7003d
:103c00002ad3bf000080fb0000004000e133210008
:103c100060c0780036f3b700bcd2bf003653e30073
:103c20002500360035d3bf003453e30021003200b5
:103c300040c8b30038f3b70035d3bf0039f3b7003d
:103c40003a73ef006f02070040c9b30038f3b700c2
:103c500034d3bf0039f3b70036d3bf003af3b7000f
:103c60006802070034d3bf0035f3b70071968000b7
:103c700040062000808f50000e00340040c9b30081
:103c800038f3b700c2002000209680001100090020
:103c90000280d800010678004036220060407e0095
:103ca00039f3b700f0c7b300ce52b6003af3b7000d
:103cb00054020700130037003553e20007003600b6
:103cc00040c8b30038f3b70035d3bf0039f3b700ad
:103cd0003a73ef004b0207003573ef00ca32af00b2
:103ce0000800370040c9b30038f3b700e0c7b3009d
:103cf00039f3b700f0c7b3003af3b7004102070049
:103d0000ca32a80001002000f012af001140b0003c
:103d1000cc52af001140b1001d003200cc52a800bf
:103d2000f012ae00cc52a9007298800083988000f7
:103d30000000200001002400e3f107000b003d001b
:103d4000ca12af000800370040c9b30038f3b7000b
:103d5000b0c7b30039f3b700f0c7b3003af3b70008
:103d600028020700ca12a80009003700ca12ae00d4
:103d70000700370040c8b30038f3b700b0c7b3003e
:103d800039f3b7003a73ef001e020700ca12a90008
:103d90000000060048baef00101a2f0050d2880029
:103da00010412e0060d2880040742d0070d288002f
:103db000f0b22c0080d2880070fc2b0090d28800da
:103dc00030502b00a0d28800a0ad2a00b0d28800cd
:103dd00030142a00c0d2880060832900d0d2880025
:103de000b0fa2800e0d28800a0792800f0d288003c
:103df000c00020005094880051948000f78f50003c
:103e00000e003e00c00020008a12b50000067800b7
:103e10000c06460080a4210060007e004100de0008
:103e2000529480004111dd0081a421000101410074
:103e3000000978008a32ec00efff39008001200091
:103e4000509488005194800030022000808f5000f0
:103e50000e003e00800120008a12b50000067800a6
:103e60000c06460080a4210060007e004200de00b7
:103e7000529480004111dd0081a421000101410024
:103e8000000978008a32ec00eeff39004002200081
:103e90005094880051948000f0022000808f5000e0
:103ea0000e003e00400220008a12b5000006780095
:103eb0000c06460080a4210060007e004300de0066
:103ec000529480004111dd0081a4210001014100d4
:103ed000000978008a32ec00eeff39000003200070
:103ee0005094880051948000b0032000808f5000cf
:103ef0000e003e00000320008a12b5000006780084
:103f00000c06460080a4210060007e004400de0014
:103f1000529480004111dd0081a421000101410083
:103f2000000978008a32ec00eeff3900c00320005f
:103f3000509488005194800070042000808f5000bd
:103f40000e003e00c00320008a12b5000006780073
:103f50000c06460080a4210060007e004500de00c3
:103f6000529480004111dd0081a421000101410033
:103f7000000978008a32ec00eeff3900800420004e
:103f8000509488005194800030052000808f5000ac
:103f90000e003e00800420008a12b5000006780062
:103fa0000c06460080a4210060007e004600de0072
:103fb000529480004111dd0081a4210001014100e3
:103fc000000978008a32ec00eeff3900007a210007
:103fd00080d78800f073210090d78800f06d210011
:103fe000a0d7880000682100b0d788004062210077
:103ff000c0d78800805c2100d0d78800e05621001f
:10400000e0d7880060512100f0d78800f04b2100f4
:1040100000d888009046210010d888005041210027
:1040200020d88800203c210030d88800103721009b
:1040300040d888001032210050d88800202d21005f
:1040400060d888004028210070d888008023210093
:1040500080d88800d01e210090d88800301a210016
:10406000a0d88800a0152100b0d888002011210018
:10407000c0d88800c00c2100d0d88800700821006a
:10408000e0d8880020042100f0d88800f0ff20004c
:1040900000d98800d0fb200010d98800c0f720008c
:1040a00020d98800d0f3200030d98800e0ef20002c
:1040b00040d9880000ec200050d9880030e820006a
:1040c00060d9880070e4200070d98800c0e020002a
:1040d00080d9880020dd200090d9880090d9200068
:1040e000a0d9880010d62000b0d98800a0d2200026
:1040f000c0d9880040cf2000d0d98800e0cb200074
:10410000e0d98800a0c82000f0d9880060c5200050
:1041100000da880030c2200010da880010bf2000ca
:1041200020da880000bc200030da88000000060099
:104130000059260040ca8800a0c7250050ca880040
:104140005098250060ca88004081250070ca880008
:10415000906a250080ca88003054250090ca8800e3
:10416000303e2500a0ca880090282500b0ca8800eb
:1041700050132500c0ca880060fe2400d0ca880001
:10418000c0e92400e0ca880080d52400f0ca880075
:1041900090c1240000cb8800f0ad240010cb880033
:1041a000a09a240020cb8800a087240030cb880070
:1041b000f074240040cb88009062240050cb88002b
:1041c0008050240060cb8800b03e240070cb880073
:1041d000302d240080cb8800f01b240090cb880079
:1041e000000b2400a0cb880050fa2300b0cb88003d
:1041f000e0e92300c0cb8800c0d92300d0cb8800e1
:10420000e0c92300e0cb880040ba2300f0cb88004f
:10421000e0aa230000cc8800c09b230010cc8800bb
:10422000e08c230020cc8800307e230030cc880036
:10423000d06f230040cc8800a061230050cc8800c0
:10424000b053230060cc8800f045230070cc880078
:104250007038230080cc8800202b230090cc88006d
:10426000101e2300a0cc880040112300b0cc880091
:1042700090042300c0cc880020f82200d0cc880015
:10428000e0eb2200e0cc8800d0df2200f0cc8800f8
:10429000f0d3220000cd880050c8220010cd880045
:1042a000d0bc220020cd880080b1220030cd880013
:1042b00070a6220040cd8800809b220050cd88004f
:1042c000c090220060cd88002086220070cd88003a
:1042d000c07b220080cd88008071220090cd8800b4
:1042e00060672200a0cd8800805d2200b0cd8800ec
:1042f000c0532200c0cd8800204a2200d0cd8800c3
:10430000b0402200e0cd880060372200f0cd880068
:10431000402e220000ce88004025220010ce8800ca
:10432000601c220020ce8800b013220030ce88000e
:10433000200b220040ce8800b002220050ce880020
:1043400060fa210060ce880040f2210070ce880023
:1043500030ea210080ce880050e2210090ce880013
:1043600090da2100a0ce8800e0d22100b0ce8800f3
:1043700060cb2100c0ce8800f0c32100d0ce8800e1
:10438000b0bc2100e0ce880080b52100f0ce8800ce
:1043900080ae210000cf880090a7210010cf8800b8
:1043a000b0a0210020cf8800009a210030cf8800e3
:1043b0006093210040cf8800e08c210050cf88001e
:1043c0008086210060cf88003080210070cf880077
:1043d000007a210080cf8800f073210090cf880000
:1043e000f06d2100a0cf880000682100b0cf8800c8
:1043f00040622100c0cf8800805c2100d0cf8800bf
:10440000e0562100e0cf880060512100f0cf880005
:10441000f04b210000d088009046210010d0880089
:104420005041210020d08800203c210030d088005d
:104430001037210040d088001032210050d0880071
:10444000202d210060d088004028210070d08800f5
:104450008023210080d08800d01e210090d08800c9
:10446000301a2100a0d08800a0152100b0d088000b
:1044700020112100c0d08800c00c2100d0d08800bd
:1044800070082100e0d0880020042100f0d08800ce
:10449000f0ff200000d18800d0fb200010d1880060
:1044a000c0f7200020d18800d0f3200030d1880050
:1044b000e0ef200040d1880000ec200050d18800bf
:1044c00030e8200060d1880070e4200070d18800be
:1044d000c0e0200080d1880020dd200090d188003d
:1044e00090d92000a0d1880010d62000b0d188003b
:1044f000a0d22000c0d1880040cf2000d0d18800b9
:10450000e0cb2000e0d18800a0c82000f0d18800d6
:1045100060c5200000d2880030c2200010d2880080
:1045200010bf200020d2880000bc200030d28800bc
:104530000000060000c3b300413622008048780026
:1045400010c3b300513622008048780020c3b30066
:10455000613622008048780030c3b30071362200f3
:104560008048780040c3b30081362200804878003c
:1045700050c3b300913622008048780060c3b30076
:10458000a13622008048780070c3b300b136220003
:104590008048780080c3b300c1362200804878008c
:1045a00090c3b300d136220080487800a0c3b30086
:1045b000e136220080487800b0c3b300f136220013
:1045c00080487800000320005094880051948000b7
:1045d000b0052000808f500008003e00000320003e
:1045e0008a12b500800678005094800001372200be
:1045f00080f07e008a32ec00f4ff390000000600f3
:10460000ffff37008612ec0080007800f03f2000aa
:1046100000806000309488003294800041f62100d0
:1046200038d3bf0000f178008612ec0080007800db
:10463000f03f20000080600030948800f0c7b30095
:104640003953b6000080fb003294800041f621000f
:1046500000f178008612ec0080007800f03f200026
:104660000080600030948800f0c7b3003a53b60071
:104670000080fb003294800041f6210000f17800b8
:10468000000006008612ec0080007800f03f200059
:1046900000806000309488003294800041f6210050
:1046a0003bd3bf0000f178008612ec008000780058
:1046b000f03f20000080600030948800f0c7b30015
:1046c0003c53b6000080fb003294800041f621008c
:1046d00000f17800000006003d13af0014aea80002
:1046e0003d13ae0014aea9003d33af00140ea80078
:1046f0003d33ae00140ea9003d53af00142ea800a8
:104700003d53ae00142ea9003d73af00042ea80047
:104710003d73ae00042ea90010c0b3003d93ae005f
:1047200000c0b3000000a700028ea9000000a60090
:08473000028ea8000000060043
:020000040000fa
:10473800741200000e0000008000000082120000c9
:104748006c00000080000000ee1200002c00000049
:10475800800000001a130000240000008000000000
:104768003e1300000a08000080000000481b0000fb
:104778001c00000080000000641b00006c080000a2
:084788008000000000000000a9
:00000001FF
